:1000000020C500003BC5000039C500000C94A22D9E
:1000100035C5000033C5000031C500002FC5000004
:100020002DC500002BC500000C947D2A0C94652B77
:100030000C94CC1923C5000021C500001FC5000089
:100040001DC500001BC5000019C5000017C5000034
:1000500015C500000C94592A11C500000FC50000F9
:100060000DC500000BC5000009C5000007C5000054
:1000700005C5000003C5000001C50000FFC4000065
:10008000FDC40000FBC40000F9C40000F7C4000078
:10009000F5C40000F3C40000F1C40000EFC4000088
:1000A000EDC40000EBC40000E9C400000660FF09D5
:1000B00061A1010962150026FF00952075088102E3
:1000C0000963150026FF00952075089102C00501FF
:1000D0000906A101050719E029E715002501950882
:1000E000750181029501750881010507190029FF35
:1000F000150026FF009506750881000508190129DD
:10010000051500250195057501910295017503916D
:1001100001C009024200020100A0FA090400000126
:10012000030101000921110100012244000705819A
:100130000308000109040100020300000009211165
:1001400001000122220007058203200001070503A8
:10015000032000011201000200000008D8042DEB6A
:100160000001010200010E034C0069006C007900DF
:1001700035003800000010036C0069006C00690055
:1001800075006D00730000000403090446001E00A2
:100190001F00200021002200290014001A0008007E
:1001A000150017002B0004001600070009000A00C4
:1001B00000571D001B000600190005000000E300A9
:1001C000E000777C2C0034004C002700260025003E
:1001D000240023002A00130012000C0018001C0049
:1001E0002F0033000F000E000D000B00E50038005B
:1001F00037003600100011000000E700E600787CB0
:10020000280032003A003B003C003D003E003F0029
:1002100001001E021F02200221022202010014140A
:100220002D005700000000000100351435022D1488
:100230005500000000000100010001000100010064
:1002400045004400430042004100400001002702F5
:10025000260225022402230200000000000064029E
:100260006400350001002E02341430142D022E00DB
:100270000000010001000100010001000100000078
:10028000000000000000000001000000000052001B
:1002900000004A0001000000500051004F004D00D6
:1002A000010000000000000000000000000001004C
:1002B0000100010001000100010022026100600054
:1002C0005F000000010055005E005D005C00000062
:1002D000570024025B005A00590000005600270214
:1002E000370036006200000000000100010001003C
:1002F00001000100010000000000000000000000FB
:100300000100000000000000000042780100457874
:10031000477849784B7843780100467848784A789E
:100320004C78000000000100010001000100010004
:1003300000000000000000000000000000000000BD
:100340000000000000000000007C000050090000D8
:100350005009000000000000AB00AE00AC0000003F
:1003600000000100010001000100010000AE00AF2B
:100370000001010101010101010102020202020268
:10038000020202030303030303030304040404043B
:100390000404050505050506060606060707070702
:1003A0000708080808090909090A0A0A0B0B0B0CB7
:1003B0000C0C0D0D0D0E0E0E0F0F0F101011111154
:1003C00012121313141415151616171718181919D5
:1003D0001A1A1B1B1C1D1D1E1E1F2020212222233A
:1003E0002424252626272829292A2B2C2D2D2E2F7B
:1003F00030313232333435363738393A3B3C3D3E92
:100400003F404142434445464748494A4C4D4E4F80
:1004100050515354555658595A5B5D5E5F61626442
:10042000656668696B6C6D6F7072737577787A7BCF
:100430007D7E8082838587888A8C8E8F9193959626
:10044000989A9C9EA0A2A3A5A7A9ABADAFB1B3B546
:10045000B7BABCBEC0C2C4C6C9CBCDCFD1D4D6D822
:10046000DBDDDFE2E4E7E9EBEEF0F3F5F8FAFDFFC0
:1004700000DA0281FFD9F1DB20A4A62EAF00A0C0D4
:10048000D30000A1C8D30000AED580A81F408D14B2
:10049000200000000000FC020202028242428202AE
:1004A000C242424202C242424202020202FC000036
:1004B000000000000000FF000000000F10100F00FF
:1004C0001F020200001F02020000000000FF0000E7
:1004D0000000000000000102020202020202020209
:1004E00002020202020202020202020202010000F1
:1004F000000000000000007C8282824400F8242278
:1005000024F800FE1212120C004C92929264000029
:1005100000000000000000000000000000000000DB
:1005200000000000000000000000000000000000CB
:10053000000000000000FCFEFEFEFE7E3E9E9E3E91
:100540007EFE1E1EFEFE1E1EFEFEFEFEFEFC0000C9
:10055000000000000000FFFFFFFFFFF0E0CFCFE052
:10056000F0FFC0C0FCF9C0C0FFFFFFFFFFFF0000AD
:10057000000000000000010303030303030303035F
:100580000303030303030303030303030301000043
:10059000000000000000007C8282824400F82422D7
:1005A00024F800FE1212120C004C92929264000089
:1005B000000000000000000000000000000000003B
:1005C000000000000000000000000000000000002B
:1005D00000000000000000000000FF01010101F127
:1005E000919191610101010101FF000000000000F3
:1005F00000000000000000000000FF808080808F6D
:10060000808182848880808080FF0000000000005C
:1006100000000000000000000000FF01010101F1E6
:10062000010101010101010101FF000000000000C2
:1006300000000000000000000000FF808080808F2C
:10064000888888888080808080FF0000000000000B
:10065000000000000000000000000000000000009A
:10066000000000000000000000000000000000008A
:100670000000000000000C0A09894929190981417C
:100680002111C93F0F010131190F844221110905C0
:100690000301C0A09088848281909894929190F0F8
:1006A000FC838080E01CFC80808087F800000000D4
:1006B000000080808080808080808080808080803A
:1006C000808080808080808080808080808080802A
:1006D000808000000000000000000000000000001A
:1006E000000000000000000000000000000000000A
:1006F0000000000000007E0F00D4FFFFFFC70000D5
:10070000007800000000000000002A2B28000000F4
:1007100000000000000000000000000000290000B0
:1007200000002C1E3420212224342627252E362D8D
:100730003738271E1F202122232425263333362E27
:1007400037381F0405060708090A0B0C0D0E0F1099
:100750001112131415161718191A1B1C1D2F3130DE
:10076000232D350405060708090A0B0C0D0E0F1082
:100770001112131415161718191A1B1C1D2F3130BE
:10078000354C8142240810204080804020100824ED
:10079000428181422410080402010102040810244D
:1007A000428181C2E4F0F8FCFEFFFFFEFCF8F0E4B9
:1007B000C2818143270F1F3F7FFFFF7F3F1F0F270E
:1007C000438101020408102040808040201008046A
:1007D00002010103070F1F3F7FFFFF7F3F1F0F072E
:1007E00003018040201008040201010204081020C7
:1007F000408080C0E0F0F8FCFEFFFFFEFCF8F0E077
:10080000C08000000000000000005F000000000742
:1008100000070000147F147F1400242A7F2A12008E
:10082000231308646200364956205000000807036D
:100830000000001C224100000041221C00002A1C74
:100840007F1C2A0008083E08080000807030000065
:100850000808080808000000606000002010080474
:1008600002003E5149453E0000427F40000072496F
:10087000494946002141494D33001814127F1000A8
:100880002745454539003C4A494931004121110974
:100890000700364949493600464949291E000000EB
:1008A0001400000000403400000000081422410041
:1008B00014141414140000412214080002015909F0
:1008C00006003E415D594E007C1211127C007F49AA
:1008D000494936003E41414122007F4141413E00AD
:1008E0007F49494941007F09090901003E414151C1
:1008F00073007F0808087F0000417F41000020400E
:10090000413F01007F08142241007F4040404000E9
:100910007F021C027F007F0408107F003E4141419E
:100920003E007F09090906003E4151215E007F0912
:100930001929460026494949320003017F01030075
:100940003F4040403F001F2040201F003F403840B4
:100950003F00631408146300030478040300615922
:10096000494D4300007F414141000204081020002E
:10097000004141417F000402010204004040404028
:1009800040000003070800002054547840007F28EE
:1009900044443800384444442800384444287F0004
:1009A00038545454180000087E09020018A4A49C6E
:1009B00078007F080404780000447D400000204057
:1009C000403D00007F102844000000417F400000AF
:1009D0007C04780478007C0804047800384444449B
:1009E0003800FC182424180018242418FC007C0863
:1009F0000404080048545454240004043F442400D0
:100A00003C4040207C001C2040201C003C403040EA
:100A10003C004428102844004C9090907C00446492
:100A2000544C4400000836410000000077000000EC
:100A30000041360800000201020402003C26232681
:100A40003C0011241FBECFEFDAE0DEBFCDBF12E0C5
:100A5000A0E0B1E0EEE9FFE502C005900D92A83DEF
:100A6000B107D9F728E0A8EDB2E001C01D92AC377C
:100A7000B207E1F70E9407240C94652FC1CAEF92D8
:100A8000FF920F931F93CF93DF93D22F4934D8F562
:100A9000C42FC695C695C695477020E2C29FD00167
:100AA000112470E0645C784FA60FB71F60E070E01F
:100AB00028E030E0241B3109FC01E60FF71FE49128
:100AC0005D910E2F10E0FD0131977F01E02F042E84
:100AD00001C0EE0F0A94EAF75E2BF701508341152F
:100AE00071F0C93061F0F801022E02C0F595E7956A
:100AF0000A94E2F75F965C915E2B5C935F976F5F61
:100B00007F4F6D17C8F2CDB7DEB7E6E00C94E92E43
:100B10009C0191509F31B8F4832F817034FF0BC03A
:100B20008295807F31FD806232FD806433FD806874
:100B3000FB010995089531FD826032FD846033FF29
:100B4000F7CF8860F5CF80E0F3CF982F92959F7014
:100B500061F420E0982F892F8695869511F02E5FFD
:100B6000982F892F8695820F089524E0F4CF8093E3
:100B7000E10608958093E206089521E001C0220F66
:100B80008A95EAF78091E206822BF4CF21E001C03A
:100B9000220F8A95EAF7822F80959091E2068923A9
:100BA000E9CF292F9A3090F5863080F590E036E035
:100BB000239F800D911D112451E081FD54E080FDA3
:100BC000550F82FD529523E0969587952A95E1F77A
:100BD000FC01EE0FFF1FE80FF91FE054F94F20E072
:100BE00030E070E04191DF01CB01022E02C096950A
:100BF00087950A94E2F78695880B842785238427B6
:100C00008E932F5F3F4F2330310561F70895292FD1
:100C10009A3070F5863060F590E036E0239F800DC5
:100C2000911D1124682F677023E0969587952A956A
:100C3000E1F7FC01EE0FFF1FE80FF91FE054F94F39
:100C400040E050E080E0219130E0062E02C0369571
:100C500027950A94E2F72170042E01C0220F0A940E
:100C6000EAF7822B4F5F5F4F4330510561F70895DC
:100C700080E008959091E20621E030E0F90101C0A2
:100C8000EE0F8A95EAF7D90101C0AA0F6A95EAF733
:100C9000EA2B01C0220F4A95EAF7892F8E23E81329
:100CA00003C0892F822B66CF2095822F8923FBCF0B
:100CB000E091E8069091E706E91302C080E008950C
:100CC0009F0157E0E59FF0011124E751F94F518151
:100CD000561306C05081581303C05581541305C0E4
:100CE0002F5F3F4FF901E770E7CF81E008958091D2
:100CF000E8062091E706281301C008950196877041
:100D0000FACF9091E306809589238093E306282FFC
:100D1000277061F4891751F09091E50692FF06C0A3
:100D200086958695869532DF1092E3060895809524
:100D3000982F8091DE0689238093DE060895803EF9
:100D40009105D1F1C8F48133910509F481C048F4CB
:100D50008932910509F471C08A32910509F47FC086
:100D6000089589339105E1F082389105C9F0853302
:100D7000910509F45DC00895843E9105D1F148F4D0
:100D8000823E910531F1833E910541F181EE90E083
:100D90000895863E9105C1F1873E9105F1F10895D0
:100DA0002091E406237009F064C02091E50623FF3A
:100DB00014C089E290E008952091E40620FD45C02A
:100DC0003091E50630FF09C024FD24C083EE90E099
:100DD00008952091E40622FDF7CF08952091E406BE
:100DE00022FD44C03091E50630FD43C024FFF5CF1D
:100DF00011C02091E50621FFF0CF8091E40684FD2B
:100E000009C087EE90E008952091E40623FFE5CF26
:100E100024FFF7CF80E090E008952091E40623FDC1
:100E20002BC03091E50631FFE1CF84EE90E00895CC
:100E30002091E40625FFD1CFBCCF2091E40625FD0B
:100E40001EC02091E50623FFC8CF89E390E00895F6
:100E50002091E40626FFC1CF8AE290E00895209118
:100E6000E40626FFBACF81E390E0089582EE90E099
:100E7000089580EE90E0089586EE90E0089585E371
:100E800090E008959091E40692FF10C041E0282F71
:100E90002471243009F040E031E0282F28712830F7
:100EA00009F030E0431711F02CE0822793FF10C0C7
:100EB00041E0282F2471243109F040E031E0282F4F
:100EC0002871283109F030E0431711F02CE0822717
:100ED0003091E50630FF10C051E0282F21712130FC
:100EE00009F050E041E0282F2871283009F040E057
:100EF000541711F029E0822731FF10C041E0282F5C
:100F00002171213109F040E031E0282F287128318A
:100F100009F030E0431711F029E0822794FF02C066
:100F200083FD877E08950F931F93CF93DF9307DF91
:100F3000EC01D23508F03DC0D03508F0AEC0C83E57
:100F4000D105F0F4C03ED10560F4C53AD10578F47E
:100F5000C430D10530F481E0219709F080E0C82F3A
:100F6000D0E0CE01DF91CF911F910F910895CE0176
:100F70008D5C9109D0654397A0F3C0E0D0E0F1CF3C
:100F8000D03478F4D03208F09BC0CE0191509F311C
:100F9000A0F78D2F77DF082F8C2F90E0D0DE902BDD
:100FA0004FC08C2F90E0CBDEDF70C82FD92BD06ADA
:100FB000D8CFC03882E5D807B8F5C03682E5D80763
:100FC00008F051C0C03482E5D807C8F4C03282E5C9
:100FD000D80708F042C08C2F8695869520E2829F24
:100FE000C0011124C37021E030E002C0220F331F82
:100FF000CA95E2F7E901C82BD92BDD68B2CF8C2F57
:1010000086958695877020E2829FC0011124C37067
:1010100021E030E002C0220F331FCA95E2F7E90158
:10102000C82BD92BDC689DCFC03C82E5D80750F493
:101030008C2F8F71C03AD24558F5982F84EF906A63
:10104000EC018FCFCE01805C9245809708F095CF60
:10105000DC2FDF71C0EFD06A84CF8C2F8F71D82F37
:10106000C1EFD06A7ECF8C2F86958695877020E25F
:10107000829FC0011124C37021E030E002C0220F22
:10108000331FCA95E2F7E901C82BD92BDA6869CF7B
:10109000F9DEC0E0D82FD06264CF8C2F8F71F2DEE2
:1010A00093E0CC0FDD1F9A95E1F7DF70282F84FFC6
:1010B00004C090E1899F90011124C22FD06951CFC3
:1010C0008D2F8F71DFDE082F8C2F90E038DE902B74
:1010D000EC01E1CF80E00895F894E82FE295EF70FD
:1010E000F0E041A18F7021E001C0220F8A95EAF75C
:1010F000922F9095942391A392A1822F892B82A362
:1011000078940895CF92DF92EF92FF921F93CF933E
:10111000DF93462F172FE82FF0E0E059FC4F7111B5
:101120000CC0E4918E2F7E2F6E2FDF91CF911F91F7
:10113000FF90EF90DF90CF900895F491EF2F86E02D
:10114000689FE00111242FEF30E0CE01B9010E9429
:10115000AD2EDB01CA01880F991F65E56A9FA001CA
:101160006B9F500D1124841B482F440F480FC90159
:10117000811B9109F89F7001F99FF00C11248F2DAC
:10118000149FB0011124672F70E06901C61AD70AB5
:10119000B601F69F6001F79FD00C1124A330B10572
:1011A00049F1B901641B7109AB01149FB001159F8E
:1011B000700D1124672F70E0261B370BF29FA001E2
:1011C000F39F500D1124752FCC3FD34050F4A13024
:1011D000B105A1F0129709F0A7CFEF2D852F7F2F32
:1011E000A3CFA430B10569F0169709F49DCF7F2DE8
:1011F0008D2D9ACF7D2DEF2D8F2F96CF7F2FED2D1B
:1012000093CFE52F7F2DF8CF9C0180E090E0269FC3
:10121000020E811D369F800D911D1124830F911D9B
:10122000089540910C0150910D0125E038E0429F56
:10123000C001439F900D529F900D1124875E994CE1
:1012400080930C0190930D01890F0895982FE82F3A
:1012500096FDE0958E2F8F7096FD8F5FE695E69553
:10126000E695E670F0E0E257FD4F2181289F202DA2
:10127000812D112422952F708295807F282B8081CB
:10128000820F97FD8195805808951F93CF93DF9328
:10129000EB01182F822F8695D9DF805887FD819525
:1012A000880F282F219F020E20E0211D1124822F5C
:1012B000BE01DF91CF911F910895622F0895E42F11
:1012C000F0E0EE0FFF1FE454FE4F6081621B0895B3
:1012D0000F931F93022F50E0FA01EE0FFF1FE0580B
:1012E000FE4FE5ADE052E7FDE195440F551F445434
:1012F0005E4FDA012C91201B310B2E0F620F1F91D4
:101300000F9108950F931F93A02FB0E0FD01EE0FF2
:10131000FF1FE058FE4F05AD0052110B2003F001F6
:10132000219FF00D1124AA0FBB1FA454BE4F2C9176
:101330002057330B4203D001439FB00D11249F016E
:101340002A0F3B1F12F421583F4F220F232F221F39
:10135000330B620F1F910F9108959091EB03982B1F
:101360009093EB030895A7C108951F93CF93DF9344
:10137000C82FD0E0FE01E85BFD4F808190910A010B
:10138000892389F04EDF182F4CDF20E8829FC001AF
:101390001124792F7158612F80913506B3DE472FC4
:1013A000282FCE01E0DFDF91CF911F9108958EC1EC
:1013B0000895982F990F990F890F982F9B5F973455
:1013C00008F096E40895EF92FF920F931F93CF9346
:1013D000DF937C0180910901ECDFC82F192F609108
:1013E00036066695669521E0620F08F46FEF8091EE
:1013F000E7039091E80308DF082FD0E0C11748F019
:1014000081E0163408F080E0CDB7DEB7E6E00C945A
:10141000E92EFE01E85BFD4F808190910A0189234E
:1014200079F0609133067091340680913506202F53
:101430004C2FF701099566DE472F282FCE0193DF49
:101440002196DCCF9091320621E0922790933206CC
:101450001092080182CF80913206837011F41092AD
:101460000801809132068C7F816080933206089556
:1014700080913206837011F010920801809132063B
:101480008C7F80933206089590913206937091F08C
:10149000811589F0893088F48F73880F880F982F11
:1014A000209132062370922B9093320610920801FD
:1014B000862F53CF089581E0F0CF88E0EECF809162
:1014C0003206869586958F5F893008F081E061E06D
:1014D000DBCF8091320686958695815009F488E0AD
:1014E00061E0D2CF90913206937059F08093330629
:1014F00060933406493708F048E740933506822F59
:101500002CCF0895E2E3F6E0818190E021E0438171
:1015100062810896E7CFE2E3F6E0818121E0438132
:1015200062818850990BDECFE2E3F6E0628120E130
:10153000620F08F46FEF818121E0438190E0D2CF08
:10154000E2E3F6E0628120E1621B08F460E0818161
:1015500021E0438190E0C6CFE2E3F6E0438120E161
:10156000420F08F44FEF818121E0628190E0BACF11
:10157000E2E3F6E0438120E1421B08F440E0818190
:1015800021E0628190E0AECF2091360630E1230F5A
:1015900008F42FEF2093360681E0DFCE2091360647
:1015A00030E1231B08F420E02093360681E0D5CEFD
:1015B000E0913706EF3F69F0E53069F0E23069F419
:1015C000EF5FF0E0E458FE4F80818093370681E0C2
:1015D000C4CEE0E0F5CFE1E0F3CFE0E0F2CFE09180
:1015E0003706EF3F91F0E53071F0E23019F0E1118C
:1015F0000EC0E3E0E150F0E0E458FE4F80818093BC
:10160000370681E0AACEE1E0F5CFE3E0F4CFE0E0F9
:10161000F2CF2091EC03382F3203C0011124923015
:1016200014F080E090E08A5D9B4F809304049093D7
:10163000050408950F931F93CF93DF93A0910404A3
:10164000B09105049D0126523440620F731F613032
:1016500042E0740710F060E072E04091280650917B
:101660002906FC0101E010E02617370748F04093F7
:10167000280650932906DF91CF911F910F9108956D
:1016800084919D91981789F0ED018A93C901C5E075
:1016900096958795CA95E1F7E80102C0CC0FDD1F4A
:1016A0008A95E2F7CE014C2B592B2F5F3F4F319695
:1016B000DBCF539A0895FC01EE0FFF1FE80FF91FCF
:1016C000E05FFC4F6183408322830895FF920F9374
:1016D0001F93CF93DF93182F062FF42EC0E0D0E096
:1016E0002F2D402F612FCE01E6DF2196C634D10584
:1016F000B9F7CDB7DEB7E5E00C94EA2EFC01AC01FA
:101700004B5F5F4F8FEF61E39191892728E030E0D5
:10171000982F990F87FF09C0892F862721503040C5
:10172000B9F7E417F50781F70895892FF7CF8111ED
:1017300044C0E9EFF2E020E030E047E0429FC00122
:10174000439F900D1124DC01A250BD4F5C9153FFCB
:1017500006C05681511103C087509D4F08952F5FD9
:101760003F4F37962330310549F7611531F18091AC
:10177000FE0283FF1CC08091050383FF1BC0809184
:101780000C0383FD1AC082E090E027E0289FF0015F
:10179000299FF00D1124CF0187509D4FDC01169633
:1017A0001C92E250FD4F208128602083089580E044
:1017B00090E0EBCF81E090E0E8CF80E090E008950A
:1017C0004115510511F0FA01099508958091AE0671
:1017D000811103C0809184060895E091B606F091CE
:1017E000B706309739F00190F081E02D309711F075
:1017F0000995089580E008959C01FC01329680E0EF
:101800009FEF4081461759F031969F3F19F44111DF
:1018100001C0982F8F5F8630A1F79F3F09F408958C
:10182000290F311D97FD3A95F90162830895FC0156
:10183000329608962191261302C0DF011E92E81706
:10184000F907C1F7089580910F0108952FB7F89413
:101850006091F5027091F6028091F7029091F80282
:101860002FBF08958091AE06811539F0EFDF462F26
:10187000572FBC01CB01BA010895E8DFDC01CB0191
:101880004091B0065091B1066091B2067091B306D6
:10189000480F591F6A1F7B1FEDCF87E797E780939B
:1018A00000089093010888E19AE00FB6F894A89593
:1018B000809360000FBE90936000FFCF089508955D
:1018C0000895FC012091EB023091EC0226173707B6
:1018D00048F06115710529F49091E8009E77909386
:1018E000E8009B0190E02115310541F4911106C0FB
:1018F0008091E80082FF32C080E0089580913A062E
:101900008115C1F18530C1F18091E80083FD30C0BF
:101910008091E80082FDECCF8091E80080FFE3CF6A
:101920008091F3004091F200582F2115310519F0F4
:101930004830510558F091E04830510509F090E0E9
:101940004091E8004E774093E800CDCF819180939D
:10195000F100215031094F5F5F4FE7CF80913A0688
:10196000811541F0853041F08091E80083FFC0CFC0
:1019700081E0089582E0089583E00895982F909380
:10198000E900891771F07091EC002091ED00509101
:10199000F00021FD09C09F5F973089F78093E9002F
:1019A0000895762F242F50E03091EB003E7F309346
:1019B000EB003091ED003D7F3093ED003091EB0076
:1019C00031603093EB007093EC002093ED00509366
:1019D000F0002091EE0027FDDECF08958091E50212
:1019E00087FF13C08091E80082FF06C08091E80065
:1019F0008B778093E800089580913A068111F2CFA9
:101A0000089580913A068115D9F38091E80080FF0E
:101A1000F8CF8091E8008E77ECCF2091E4003091F0
:101A2000E50095E6A9012091EC00822F817020FF4E
:101A300006C08091E80080FF06C080E008952091F4
:101A4000E80022FD1AC080913A06811589F08530A0
:101A500089F08091EB0085FD0FC02091E40030916A
:101A6000E50042175307F9F29150E1F684E008953A
:101A700082E0089583E0089581E00895CF93DF9395
:101A8000C8EDD0E088818F7E8883E7EDF0E080812B
:101A90008160808384E082BF81E08093E40288815A
:101AA0008E7F8883E2EE10821092DA00A1EEB0E021
:101AB0001C9288818F778883888180688883888159
:101AC0008F7D888319BC10923A061092E30210921F
:101AD000EE031092E202A0EE8C918B7F8C938881B2
:101AE0008160888342E060E080E048DFA1EEB0E002
:101AF0008C918E7F8C93E2EEF0E080818160808318
:101B0000808188608083E0EE80818E7F8083888101
:101B100080618883DF91CF910895E8EDF0E08081C6
:101B20008E7F80831092E2001092DA001092E10022
:101B3000A0EEB0E08C9181608C9380818F77808360
:101B400019BCA7ED8C918E7F8C9380818F7E8083D2
:101B50001092E4020895A0E0B0E0E1EBFDE00C9407
:101B6000C72ED82E809178018D1549F000913A0743
:101B700010913B070115110539F4D0927801CDB7CA
:101B8000DEB7ECE00C94E32E8D2D0E94A505B82E57
:101B90009091390780E0891781F3F8012081B2160E
:101BA00009F455C08F5F0B5F1F4FF5CFF80101801F
:101BB000F281E02DEE0DFF1D2081822F81568A31AA
:101BC000B8F420522052330B46E0429FC001439F9D
:101BD000900D112425E0492D62E08E5F974F0E9401
:101BE0003F058FEFE81AF80A892D865F982E65C0A9
:101BF000203240F720E2E6CFED120FC0A814B9045E
:101C000001F582ED97E020E14C2F60E10E943F0555
:101C10008FEFE81AF80AC85F6CC0C7010197A816D1
:101C2000B90691F082EA97E0AE14BF0461F31F3F5A
:101C300029F082E897E0AE14BF042CF382E997E024
:101C4000E2CF82EC97E0DFCF82EB97E0DCCF8181BF
:101C50009281892B09F491CFD0913807D11509F4DD
:101C60008CCFECE3F7E080E491E011920197E9F783
:101C7000F801A181B281FD0101900020E9F73197BF
:101C8000EA1BAE2ECD2EC3944AE04E9F402D112468
:101C9000425080E590E09C01241B3109A901559533
:101CA0004795942E2C2D220F220F220F821B910973
:101CB00095958795C82FE12CF12CEA1408F476CF7E
:101CC000E8E2F7E010E0A081B181109719F08C9163
:101CD0008B1529F032961F5F1D13F5CF1FEFE12CF6
:101CE000F12CA12EB12EBB0CBB088D2F8150990B6E
:101CF0004C01EC1408F041CFE1107ECF82EF97E069
:101D0000111509F480CF82EE97E07DCFA0E0B0E01E
:101D1000ECE8FEE00C94C92E7C016B015A01809125
:101D200091060AE010E08A3010F001E010E0C1E016
:101D3000D0E0B601C701F5010995811115C02196C2
:101D40000C171D078CF0CC9F9001CD9F300D300DEE
:101D5000112480E090E045E34A95F1F700000196F8
:101D600082179307C1F7E5CFCDB7DEB7EAE00C9451
:101D7000E52E3BB1377F2BB128604FB7F89480E157
:101D800093E0FC010196508168E02BB9000000C08F
:101D900057FF3BB9550F000000C000C000C03BB961
:101DA00000C06A9591F753E0823E950751F74FBF07
:101DB0008FE594E00197F1F700C0000008950F93BC
:101DC0001F93CF93DF93EB018A0190913A069430F1
:101DD00059F58093E9008FEF9091E80095FD06C0DA
:101DE00095ED9A95F1F700008150B1F78091E800E8
:101DF00085FF1AC012DE811112C08091E80085FDB6
:101E000006C08091E8008E778093E800F3CF888148
:101E10008093F1000150104011F02196EECF809197
:101E2000E8008E778093E800DF91CF911F910F91AA
:101E30000895603229F440E250E0BC0182E0BFCF57
:101E40000895CF93DF93EC0148E050E0BC0181E0BE
:101E5000B6DF88E0FE01ADEEB2E001900D928A950A
:101E6000E1F7DF91CF9108959091E50692FB22274B
:101E700020F9281779F080FB92F99093E50660919C
:101E8000E4067091E50684E090E00E94612F82E014
:101E90000C94810608951F93CF93DF93122F863001
:101EA000E0F46A30D0F44630C0F4C42FD0E0CC0F58
:101EB000DD1F2CE0629FC00DD11D112498E7899F82
:101EC000C00DD11D1124632FCE0189960E94472F8A
:101ED000612FCE018A960E94472FDF91CF911F91EB
:101EE0000895AF92BF92CF92DF92FF920F931F930C
:101EF000CF93DF93A12CB12CC0E06501D0E018C0D6
:101F000021E030E0C43020F4F801859195919C01E6
:101F10004F2D6D2F8C2FBFDFF3940E5F1F4F8F2D32
:101F2000863071F7DF5F86E0C80ED11CDA3039F0F9
:101F30008601000F111F04571E4FF12CE1CFCF5F18
:101F40008CE3A80EB11CC630C1F6DF91CF911F9172
:101F50000F91FF90DF90CF90BF90AF900895809148
:101F6000DE069091E606892B9091DF06911589F0A7
:101F7000892B90E02CED32E0F90140812F5F3F4F3B
:101F800041119F5F42E0223E3407B1F79111109258
:101F9000DF068093DA0248E050E068EB76E08AEDF5
:101FA00092E00E94052F892BB9F088E0EAEDF2E07B
:101FB000A8EBB6E001900D928A95E1F7E091B606A4
:101FC000F091B706309741F00280F381E02D309711
:101FD00019F08AED92E0099508951092DE06ECED75
:101FE000F2E086E011928A95E9F71092E606B7CF03
:101FF000F4DF88E19AE00FB6F894A895809360002A
:102000000FBE90936000FFCFAAE2B0E0EAE0F0E1FB
:102010000C94D02E85EE92E0FC0101962091F10007
:10202000208322E08D3E9207B9F78091E602893045
:1020300009F457C0C8F4823009F4B2C0833009F4FF
:1020400082C0813081F18091E80083FFE6C08091F9
:10205000E5029091E6029A3008F0DFC0E92FF0E047
:10206000E959F04D0C94F82E8A3009F489C08B3070
:1020700051F78091E502813231F78091E902909128
:10208000EA02892B01F78091E800877F8093E800BE
:10209000A5DC81E09091E702911101C080E080937E
:1020A00010019BDFD0CF8091E502813A61F68091EB
:1020B000E800877F8093E8008091E9029091EA022E
:1020C000892B59F060E080E090E070E0FADB8091CD
:1020D000E8008B778093E800B6CF68E08DEE92E061
:1020E000F4CF8091E502813209F0ADCF8091E90211
:1020F0009091EA02892B09F0A6CF8091E800877FB2
:102100008093E8008091E80082FF18C02091F300DE
:102110008091F200922F029731F48091F10081308A
:1021200011F0863021F48091F10080930F018091AD
:10213000E8008B778093E80051DC85CF80913A06E8
:102140008111E0CF80CF8091E502813A09F07BCF09
:102150008091E9029091EA02892B09F074CF809175
:10216000E800877F8093E8008091E80080FFFCCF43
:10217000809110018093F1008091E8008E77DACF92
:102180008091E502813209F05ECF8091E800877F7F
:102190008093E80023DC8091E80280930E0153CF06
:1021A0008091E502813A09F04ECF8091E800877F67
:1021B0008093E8008091E80080FFFCCF80910E01C1
:1021C000D9CF803889F0823841F58091E9028F704B
:1021D000873018F58093E9008091EB0085FB882714
:1021E00080F91092E90006C08091EE03880F90916B
:1021F000E202892B9091E800977F9093E80080930A
:10220000F1001092F1008091E8008E7723C08111D7
:1022100016C08091E702813009F18091E80083FFC8
:102220000AC08091E800877F8093E8008091EB00EE
:1022300080628093EB00AA96E3E00C94EC2E82304F
:1022400061F78091E702811579F01092E9008091A1
:10225000E800877F8093E800C1DBDFCF933009F08F
:1022600080E08093EE03F1CF8091E9028F70282FF8
:102270002150263090F68093E9002091EB0020FF5A
:10228000E4CF933031F48091EB0080628093EB00D7
:10229000DCCF9091EB0090619093EB0021E001C0C6
:1022A000220F8A95EAF72093EA001092EA008091C3
:1022B000EB008860EBCF8111B0CF8091E7028F7780
:1022C000182F8091E3008078812B8093E300809128
:1022D000E800877F8093E80081DB8091E80080FF41
:1022E000FCCF8091E30080688093E30083E01111CC
:1022F00001C082E080933A0690CF8058823008F087
:102300008CCF2091E7023091E8022C3D83E0380722
:1023100089F583E08A838AE289834FB7F894DE01E6
:10232000139620E03EE051E2E32FF0E05093570097
:10233000849120FF03C082958F703F5F8F708A3039
:10234000B8F0895C8D931D922F5F243169F74FBFE0
:102350008091E800877F8093E8006AE270E0CE0118
:102360000196AFDA8091E8008B778093E80055CF33
:10237000805DE8CF832F90E08330910511F160F408
:102380008130910509F46BC08230910509F045CF89
:1023900082E4E2E1F1E028C02091E9023091EA0212
:1023A0008132910509F452C08232910509F035CF8E
:1023B0002130310508F45BC009F02FCFECEAF0E0E2
:1023C00013C0822F90E0213099F182309105B9F14C
:1023D000009709F022CFE8E8F1E0E4918E2FE8E8D9
:1023E000F1E0009709F419CF2091E800277F2093AE
:1023F000E8002091EB023091EC028217930708F479
:102400009C0140E021153105B1F5411134C08091A6
:10241000E80082FDA7CF80913A06811509F4A2CF8A
:10242000853009F49FCF8091E80083FFF0CF9ACFE9
:10243000E6E7F1E0E4918E2FE6E7F1E0D2CFE6E6C1
:10244000F1E0E4918E2FE6E6F1E0CBCF21303105CB
:1024500050F009F0E2CE89E0EDE3F1E0C5CF82E192
:10246000E4E5F1E0C1CF89E0E4E2F1E0BDCF84E44E
:10247000EEECF0E0B9CF80913A06811509F472CF05
:10248000853009F46FCF8091E80083FD6BCF809198
:10249000E80082FDBCCF8091E80080FFB3CF40917F
:1024A000F3008091F200942F2115310519F0883046
:1024B000910550F041E0089709F040E08091E80074
:1024C0008E778093E8009ECF44914093F10031963F
:1024D000215031090196E8CF803809F09ECE8091D5
:1024E000E800877F8093E8008091E3028093F10009
:1024F0008ACE811192CE8091E702182F823008F0A7
:102500008CCE8091E800877F8093E8001093E302EF
:1025100065DA1115B9F084E080933A0642E061EC87
:1025200081E02CDA42E261EC82E028DA42E260ECFF
:1025300083E024DA80913A06843051F482E080937B
:1025400011016BCE8091E30087FDE5CF81E0E4CF00
:1025500081E0F5CFCF93C82F811599F08450813A4F
:1025600090F4ECEDF2E082EE92E02081C217D9F017
:1025700031968E179F07C9F76C2F8AED92E03CD9F0
:10258000EEDCCF9108958C2F805E8830D0F7C77035
:1025900021E001C0220FCA95EAF78091DE06822B66
:1025A0008093DE06EDCF6C2F8AED92E040D9D7DC28
:1025B000E3CFCF93DF93EC01805E9109089720F081
:1025C00066E673E1209711F467E573E1CE010E949E
:1025D00088058C2FBFDFDF91CF910895CF93DF93D4
:1025E000EC018A81823039F4FB0182819381E1DF41
:1025F0008D8182608D83DF91CF910895FB01808171
:102600009181D7CF811549F0982F9450913A30F4A9
:10261000682F8AED92E00BD9A2CC0895982F905E96
:102620009830D8F7982F81E091FD84E090FD880FD5
:1026300092FD82950E949706EFCFCF93DF93EC0136
:10264000E1DFCE01805E9109089720F06FE673E12B
:10265000209711F460E673E1CE010E948805DF91B6
:10266000CF910895FC018281813029F4FB018081A2
:102670009181E3CF08958230E9F7FB018281938154
:10268000F8CF1F93CF93DF93182FEB0163DF2097D1
:1026900031F4812FB7DFDF91CF911F9108958FE93A
:1026A0009FE00197F1F700C000002197F0CF81155E
:1026B00031F09091DE06982B9093DE0650CC089571
:1026C000811519F00E9497064ACC0895811531F0C2
:1026D0009091E606982B9093E60641CC08958115DB
:1026E00039F080959091E60689238093E60637CCF1
:1026F0000895CF93DF93EB01FC0144815581608500
:102700007185CE015DD89B8190958091E6068923E5
:102710008093E6068C810E94970621DC87E019925F
:102720008A95E9F7DF91CF9108950F931F93CF9387
:10273000DF938C01EB018D8181FD16C082608D835A
:102740008091E6069B81892B8093E6068091DE06C8
:102750009C81892B8093DE0602DCF8014281538143
:1027600060857185CE012CD81092D8061092D906BA
:102770008D8180FD03C0BE01C801BBDFDF91CF9119
:102780001F910F910895CF92DF92EF92FF921F93C6
:10279000CF93DF9300D000D0CDB7DEB7C090500606
:1027A000D0905106E0905206F09053064FD8DC01CD
:1027B000CB018C199D09AE09BF0911E08436910542
:1027C000A105B10568F14ED8DC01CB010296A11D2F
:1027D000B11D89839A83AB83BC8380913F01909123
:1027E00040018F59994F20913E01422F50E02530F2
:1027F00008F044E09E012F5F3F4FB9010E94122F65
:1028000083E090E00E943F2E182F811549F01ED8DA
:10281000609350067093510680935206909353062E
:10282000812F0F900F900F900F90DF91CF911F91FC
:10283000FF90EF90DF90CF900895A0E0B0E0E3E24A
:10284000F4E10C94C72EB82EEB01A42E4901C880E8
:10285000D980EA80FB800E94260CDC01CB018C1918
:102860009D09AE09BF0984369105A105B10510F493
:10287000A11421F1EB2CFB2CFF0CFF089B2D88E011
:102880009802F0011124EA5DFE4F818192818F59F7
:10289000994F2081422F50E00217110508F4A8013A
:1028A000B4010E94122FC7010E943F2E811539F0FA
:1028B0000E94260C688379838A839B8381E0CDB74D
:1028C000DEB7ECE00C94E32E0F931F9341E0909160
:1028D00070068091E206981301C040E001E010E02C
:1028E00022EE36E06CE476E084E0A7DF811571F03B
:1028F00041E0909171068091E106981301C040E09B
:1029000021EE36E068E476E085E097DF1F910F91D5
:102910000895A1E0B0E0EFE8F4E10C94CF2E8091AF
:102920003F0689832091730690E041E0281719063D
:1029300009F440E08D019E012F5F3F4F60E476E097
:1029400087E07BDF2196E4E00C94EB2ECF92DF92C0
:10295000FF920F931F93CF93DF93F82E6B01EA0141
:10296000A801B901CE010E94052F41E0892B09F48D
:1029700040E09E01B6018F2D60DFDF91CF911F9166
:102980000F91FF90DF90CF9008950F931F9305E074
:1029900010E027E636E0AC0164E576E082E0D6DFC1
:1029A0001F910F910895A1E0B0E0E9EDF4E10C94DE
:1029B000CF2E0E94E60B898301E010E022E736E08B
:1029C000AE014F5F5F4F64E476E086E0BFDF2196A3
:1029D000E4E00C94EB2EACE0B0E0E1EFF4E10C9419
:1029E000CF2E80918D0690918E06A0918F06B0918A
:1029F000900689839A83AB83BC83809189069091EA
:102A00008A06A0918B06B0918C068D839E83AF833E
:102A1000B8878091850690918606A0918706B0912F
:102A2000880689879A87AB87BC870CE010E024E78B
:102A300036E0AE014F5F5F4F6BE376E088E086DF04
:102A40002C96E4E00C94EB2EAF92BF92CF92DF92E3
:102A5000EF92FF921F93CF93DF9300D000D000D06E
:102A6000CDB7DEB75B0180E090E00E943F2E182FCB
:102A7000811509F45FC080912901482F50E0811130
:102A800041E060912A0170912B016F59794FCE017D
:102A900006960E94122FC0905D06D0905E06E090D0
:102AA0005F06F09060060E94260CDC01CB018C19B9
:102AB0009D09AE09BF0984369105A105B10538F419
:102AC00082E696E00E947E0B9E81891799F181E053
:102AD00090E00E943F2E8115C1F180913101482F75
:102AE00050E0863008F045E060913201709133018A
:102AF0006F59794FCE0101960E94122F82E696E01F
:102B00000E947E0B9E81891320C00E94260C609338
:102B10005D0670935E0680935F069093600685E085
:102B2000FE013196A8E5B6E001900D928A95E1F795
:102B300081E00CC085E0E2E6F6E0DE01119601904E
:102B40000D928A95E1F71111EACF80E095E0E8E572
:102B5000F6E0D50101900D929A95E1F70F900F9054
:102B60000F900F900F900F90DF91CF911F91FF90DA
:102B7000EF90DF90CF90BF90AF9008950F931F9389
:102B8000CF93DF93863008F56A30F8F44630E8F4E6
:102B9000C42FD0E0CC0FDD1F9CE0699FC00DD11D7C
:102BA000112498E7899FC00DD11D1124CE0189966B
:102BB0000E942B2F082FCE018A960E942B2F902F38
:102BC000DF91CF911F910F91089580E090E0F8CFB1
:102BD000462F7A3030F4663020F4863010F4672FB8
:102BE000CDCF80E090E00895CF92DF92FF920F93D7
:102BF0001F93CF93DF936C010091E2068091E10671
:102C0000082BC5E0D0E010E0C8010C2E02C095955D
:102C100087950A94E2F780FD0CC02197A8F7F12C64
:102C20008F2DDF91CF911F910F91FF90DF90CF906B
:102C30000895FC2EB6018C2FCBDF0E9493070197DD
:102C400061F3EECF1F93CF93DF93FC012581C08109
:102C5000D181CE01211579F0611569F0C5DF182FFA
:102C6000682FCE010E94D105BE01812FB1DFDF9117
:102C7000CF911F9108950E940706182FF5CFCF938B
:102C8000DF93EC01B1DFBE01A3DF0E949307DF9168
:102C9000CF910895FC012481211599F080819181C3
:102CA000EEDF282F92959F70963099F060F4925F36
:102CB0009F70923030F4203FB1F038F481E0283E2C
:102CC00038F080E008959A5FF3CF81E0243FC9F7A0
:102CD000089591E0213F09F090E081E0283E08F05E
:102CE00080E0892B089581E00895673021E0720724
:102CF0008105910528F4CB0187509D4F0C942B2F13
:102D000080E00895CF92DF92EF92FF92CF93DF930E
:102D1000EC01C880D980EA80FB80B601C701E5DFFD
:102D20009FEFC91AD90AE90AF90AC882D982EA8248
:102D3000FB82DF91CF91FF90EF90DF90CF900895CD
:102D400085E290E00E942B2F863269F486E290E0C3
:102D50000E942B2F863039F487E290E00E942B2FBF
:102D600091E0863109F090E0892F8170089580E02C
:102D700090E00E94332F833E9E4F09F4E1CF80E024
:102D8000089548E050E067E170E082E396E00E9439
:102D9000382F1092EB03089581E1809332068091E1
:102DA000790190917A01A0917B01809333069093F1
:102DB0003406A09335068FE7809336068FEF809315
:102DC0003706DFCFA0E0B0E0E8EEF6E10C94CB2EC2
:102DD0000E94320CAB01BC014093E2035093E30329
:102DE0008093E4037093E5031091E603809108015A
:102DF000823009F4D9C1D0F4811120C010920901A8
:102E00004093E7035093E8036093E9037093EA0368
:102E100080913206837021F08091320686958695E6
:102E20008093E60381E08093080103C0833009F4B6
:102E3000C5C1CDB7DEB7E8E00C94E72E809107015D
:102E4000181325C09091320693702091060130E04E
:102E500081E09217130609F480E080930B018091C2
:102E6000370690910A01981739F080930A0140E0E3
:102E700060E080E00E94D709193058F4E12FE1505A
:102E8000E83060F4F0E0EF58F04D0C94F82E81E05B
:102E9000E4CF1F3F09F458C180E037C080910B0197
:102EA0008115D1F340E060E080E00E94D709F4CFC3
:102EB000809109010E94D909C82F092F609133061A
:102EC00070913406809135060E948208F62EE72E16
:102ED000D82ED0E00C1709F020F481E00634A8F0D9
:102EE000DBCFFE01E85BFD4F808190910A018923D1
:102EF00031F02D2D4E2D6F2DCE010E94B30921965C
:102F0000E9CF85E499E00E94E309909109019F5F70
:102F10009093090181118DCF82E080930801809107
:102F20000B01811186CF111184CF83E07CCF8DE519
:102F300099E0E9CF8FE599E0E6CF88E699E0E3CF25
:102F4000809109010E94D909C82F092F6091360686
:102F500066958091E7039091E8030E940409D82EBA
:102F6000D0E0CE01880F991F80589E4F7C010C172E
:102F700009F008F4B2CFFE01E85BFD4F808190912B
:102F80000A01892309F451C0F70144AD4057550B9C
:102F900085AD8052990B449F9001459F300D300DB7
:102FA0001124889FA001899F500D500D1124240FDA
:102FB000351F822F2230310520F19FEF213E8EE117
:102FC000380740F4C901E5E096958795EA95E1F761
:102FD000982F985F61E0462F490F5527551F55954B
:102FE0004795842F449FF001459FF00DF00D11246B
:102FF0002E173F07F8F4942F9150961760F7862FFD
:10300000815090E0BC01660F771F680F791F75959E
:1030100067956D0D70913406809135060E94820887
:10302000472F282FCE010E94B309219682E0E80E97
:10303000F11C9DCF4F3F29F3642F6F5FDECF80914E
:1030400009010E94D909C82FF92E609136066695AC
:1030500066958091E7039091E8030E940409E82EA9
:10306000805C0E9426098058D82E8E2D0E94260949
:103070008058C82ED0E0CF1520F081E09F2D9634E7
:103080002ECFFE01E85BFD4F808190910A018923DC
:1030900091F06091330670913406809135060C2FC3
:1030A0002C2D4D2D0E9482090E948208472F282F27
:1030B000CE010E94B3092196DECFC0910901C11152
:1030C0001FC06091360620E1620F08F46FEF809117
:1030D000E7039091E8030E94040965E070E00E9414
:1030E000AD2E892B69F40E94110926E4829FA0016C
:1030F0001124852F880F880B5093040180930501BC
:103100008C2F0E94D909EC0190910B01911117C0ED
:1031100020910401309105012817310590F02D17F9
:10312000310578F4822F0E94B50987E48093040169
:103130001092050106C08C2F0E94B509CF5FCD17F4
:10314000D0F381E0D634CBCE9091E803A091E9038F
:10315000B091EA03892F9A2FAB2FA6959795879563
:10316000A69597958795837090E0A0E0B0E08230B7
:103170009105A105B10589F083309105A105B1053F
:1031800079F040E060E010979040814059F464E1AC
:1031900080E00E94D70982E046CE44E160E0F8CFAB
:1031A00044E164E184E1F5CF109307018091320698
:1031B0008370809306010E94B90EB7CE8091EB0315
:1031C0008111DFDDE090E703F090E8030091E9036F
:1031D0001091EA038091AE06811579F00E94260CC9
:1031E0006E197F09800B910B653071058105910582
:1031F00008F41FCE109208011CCE0E94320CF0CFB2
:10320000A0E1B0E0E6E0F9E10C94C32EFE013196B6
:10321000DF0180E11D928A95E9F701E110E099EF65
:10322000A92E92E0B92E612C712C230153944A18D7
:103230009E2E8F2E6201730181E1481651046104B4
:1032400071041CF080E1C82ED12CA601B501892D96
:10325000982D0E94382FAC0CBD1C0D2C000C0008C2
:103260004C185D08600870080150104019F760960E
:10327000E0E10C94DF2E6FEF85E290E00E94472F93
:103280006FEF86E290E00E94472F6FEF87E290E0B9
:103290000E94472F60E088E290E00E94472F0E9442
:1032A000710FAEDF66E285E290E00E94472F66E094
:1032B00086E290E00E94472F66E187E290E00C945E
:1032C000472F63EE7EEF80E090E00E94612F60E088
:1032D00082E090E00E94472F81E08093E10661E068
:1032E00083E090E00E94472F60E074E184E090E08A
:1032F0000E94612F51DDBFDF60E070E0AB018FE025
:1033000090E00E94592F60E070E0AB0183E190E013
:103310000E94592F36CDAB0124E630E0BC0188E78E
:103320000E94762C9C0181E0232B09F080E0089517
:10333000809130068115F1F00E94260CDC01CB0152
:10334000805A9541AF4FBF4F80932A0690932B062A
:10335000A0932C06B0932D0680913F0681110AC0E0
:1033600062E070E08EE693E0D6DF811519F081E02F
:1033700080933F06089580913006811561F0809119
:103380003F06811541F062E070E08CE693E0C3DF18
:10339000811110923F0608951F921FB61F921124AB
:1033A0008F939F93AF93BF938091ED03811113C0CF
:1033B0008091F5029091F602A091F702B091F80287
:1033C0004196A11DB11D8093F5029093F602A09342
:1033D000F702B093F802BF91AF919F918F911F9028
:1033E0001FBE1F9018952FB7F8948091F502909109
:1033F000F602A091F702B091F8022FBF0895CF9383
:10340000DF93EC01F0DF8C1B9D0BDF91CF910895D2
:10341000AFE0B0E0EEE0FAE10C94C82EFE01319688
:10342000DF018AE01D928A95E9F78CECC82E82E0D4
:10343000D82E7F01AE2E9F2C07ED12E0F601819170
:103440006F018F3F09F43DC0F894E82FE295EF70CB
:10345000F0E021A18F7041E001C0440F8A95EAF7A6
:10346000922F942B91A392A1842F8095892382A3DC
:10347000789400C0E1EDF2E031E0B12C21912F3FD2
:1034800079F0A22FA295AF70A05EB0E08C9190E091
:103490002F7002C0959587952A95E2F780FFA5C009
:1034A00080E0B82A330F0E171F0741F7F60182910B
:1034B0008F3F11F00E946C0880EA8A95F1F7F701BE
:1034C000B0828FEFE81AF80A81EDC81682E0D806BC
:1034D00009F0B4CF4AE050E06A2D792D84EA96E0F5
:1034E0000E94052F009749F02AE0EA2DF92DA4EA61
:1034F000B6E001900D922A95E1F70091A30610E045
:103500000756194F892B09F472C081E08093980601
:103510006ADF80939606909397068091AE06811598
:1035200009F4BCC07E018BE0E80EF11CF70185E0D8
:1035300011928A95E9F7809191068A3008F07AC055
:1035400044E255E1B701C8010E94860E811509F4D5
:1035500094C045EC54E1B701C8010E94860E811564
:1035600009F48BC043EC53E1B701C8010E94860EF9
:10357000811509F482C044E654E1B701C8010E94F4
:10358000860E811509F479C043ED54E1B701C801F5
:103590000E94860E811509F470C049E854E1B70114
:1035A000C8010E94860E811509F467C04BEE54E1F4
:1035B000B701C8010E94860E811509F45EC0109201
:1035C00091068091950690E045E050E0B70187565E
:1035D000994F0E94052F21E020939406892B09F032
:1035E0003FC02F96EBE00C94E42E832F5ACF8091AE
:1035F0009806811509F491CFE0909606F090970611
:10360000F2DE8E199F09059708F487CF45E050E058
:1036100064EA76E0C8010E94052F892B41F085E01D
:10362000E4EAF6E0D80101900D928A95E1F7109254
:10363000980673CFC0909206D0909306D4DE8C1972
:103640009D09843F914008F07BCF809194068115BD
:1036500041F2F70185E011928A95E9F710929406FC
:10366000A0919506B0E0A756B94F85E0FE013B96C4
:1036700001900D928A95E1F7B4CF809191068F3F2A
:1036800031F4B1DE8093920690939306DECF8F5F84
:10369000809391068A3008F494CFF3CFE09095069A
:1036A000F12CC7018756994F7C0185E0F801A2E60D
:1036B000B6E001900D928A95E1F782E696E00E94CD
:1036C0007E0B8093610685E0E7E6F6E0D701019086
:1036D0000D928A95E1F7C0906C06D0906D06E0904F
:1036E0006E06F0906F068091800690918106A09101
:1036F0008206B0918306C816D906EA06FB06B1F029
:10370000C0928006D0928106E0928206F0928306F3
:103710000E94260CC61AD70AE80AF90AC092B00617
:10372000D092B106E092B206F092B3068091700694
:103730008093E206809171068093E1068091720683
:103740008093840680917306811591F1F1DD80915B
:103750007C0690917D06A0917E06B0917F064091F7
:1037600078065091790660917A0670917B060091F7
:1037700074061091750620917606309177060093B5
:103780008D0610938E0620938F06309390064093FB
:10379000890650938A0660938B0670938C068093FB
:1037A000850690938606A0938706B093880619CF66
:1037B000E2DDCDCFFF920F931F93CF93DF93C62F00
:1037C000D42FF22E8115A9F06093DC060CDE8093D5
:1037D0000E0390930F0381E0C1FD84E0C0FD880FCC
:1037E000C2FD82950E945713CDB7DEB7E5E00C9479
:1037F000EA2E8091DC06681333C000910E0310910D
:103800000F03F1DD801B910B883C910548F51D2FBE
:10381000105ECD17A1F0C77001E0802F01C0880FA6
:10382000CA95EAF70E946013183048F48D2F87700C
:1038300001C0000F8A95EAF7802F0E94571360E0BD
:1038400070E08F2D0E94411381E0D1FD84E0D0FD16
:10385000880FD2FD8295183038F60E946013C4CFCD
:1038600081E0C1FD84E0C0FD880FC2FD8295F5CFE7
:10387000A4E0B0E0EEE3FCE10C94C62E7C01FC0178
:103880008481811509F4ADC061E0C701DBD96C0109
:10389000F70185818115D1F00091D8061091D906E4
:1038A0000115110599F0C016D10689F02EE6A22E59
:1038B00021E0B22E011511F0A12CB12C60E0802F77
:1038C0000E94970BFC01892B09F03AC08601F70191
:1038D0008581811509F4EBC09801375720383105EF
:1038E00008F0E5C0003108F06DC066E071E080E0EE
:1038F00090E0FBD9811166C0A12CB12C45010111CA
:103900002FC089829A82AB82BC828E010F5F1F4FCB
:10391000C801F8D9B02EA12E813008F453C009F0A7
:103920007BC0C801EFD9813071F5C801EBD960E5E2
:1039300070E0893311F060E070E00E944113E8CF3D
:10394000858184608583C082D182BF01C5010E94C8
:1039500095131092E60661E0C70174D98C01B7CFC8
:1039600087E0881681E09806A104B10459F1B401FA
:10397000C501BBD99FEF891A990AA90AB90A811111
:10398000EFCF0150BCCF823029F4C801BBD90E94CF
:10399000AA12BECF833029F4C801B4D90E94021301
:1039A000B7CF843069F4C801ADD9C12CD12C282FF0
:1039B0002053330B2A303105C0F0C114D10411F566
:1039C0008111A6CF8091E306877059F0F7018581B8
:1039D000811539F08091E50682FF03C082E00E94E4
:1039E00081062496EDE00C94E22E4AE04C9DC00145
:1039F0004D9D900D1124280F391F69018B2D9A2D93
:103A000081D9D5CFEFE9FFE03197F1F700C0000091
:103A100091E0C91AD108D1CFE82FF0E0EE5FF84F5E
:103A20009491792E282F26952695269530E0F90138
:103A3000EE50F94FC4908770D12C082E02C0D59457
:103A4000C7940A94E2F7F901EE51F94FA490B12C12
:103A5000082E02C0B594A7940A94E2F72E52394F6B
:103A6000F9018490912C02C0959487948A95E2F78D
:103A7000C0FE03C081EE0E94AA12A0FE03C086EE23
:103A80000E94AA1260E070E0872D0E944113A0FE00
:103A900003C086EE0E940213C0FE03C081EE0E94A6
:103AA000021380FE35CF60E070E08CE246CF312F0C
:103AB000375509F07EC0A02EB12C011183CF682F9D
:103AC00080E00E94970B6C01892B09F47BCFF701F2
:103AD0008581F601958180FB90F99583811509F424
:103AE00048C081DC8093DA069093DB06F601828180
:103AF0008F5F82838091E6069091DE06892B838317
:103B00008091DF06848340916E0150916F01609136
:103B1000760170917701C6010E94E00BF601858164
:103B200081FD03C0A12C97E5B92EA092D806B092D2
:103B3000D906F7019581911509F428C41092DC0685
:103B4000980130572332310508F007C484E090E033
:103B50000E94332F8093E4069093E506F801E1502C
:103B6000F047E232F10508F04BC0E758F04D0C94F5
:103B7000F82E409174015091750160917601709119
:103B80007701C6010E94E00BF601858181FFD1CF4C
:103B9000B6018EE691E00E9479138091D80690914B
:103BA000D9068115974529F61092D8061092D906A4
:103BB000C0CFF801E851FC47E730F10508F0B9CF74
:103BC000E556F04D0C94F82E26E241EE61EEF2DD62
:103BD000F9CE27E245EE65EEFACF26E241EE60EE41
:103BE000F6CF27E245EE64EEF2CF26E241EE62EE3A
:103BF000EECF27E245EE66EEEACF28E241E0EBCFDA
:103C00008091E40681608093E4066091E4067091FF
:103C1000E50684E090E00E94612F0E94ED0FD2CE75
:103C20008091E50688608093E506EFCF8091E406F9
:103C30008260E9CF8091E4068460E5CF8091E4065C
:103C40008860E1CF8091E5068160EDCF8091E50647
:103C50008260E9CF8091E4068061D5CF8091E4064F
:103C60008062D1CF8091E4068064CDCF0E94ED0FB9
:103C70008091E4068068C7CF8091E4068C60C3CF52
:103C80008091E5068360CFCF8091E4068E7FBBCF25
:103C90008091E506877FC7CF8091E4068D7FB3CF03
:103CA0008091E4068B7FAFCF8091E406877FABCF16
:103CB0008091E5068E7FB7CF8091E5068D7FB3CFEB
:103CC0008091E4068F7E9FCF8091E4068F7D9BCF0D
:103CD0008091E4068F7B97CF0E94ED0F8091E406E0
:103CE0008F7791CF8091E406837F8DCF8091E50619
:103CF0008C7F99CF9091E406892F8B7F92FF84600F
:103D0000877F92FF88607FCF8091E506982F9095FE
:103D100090FB80F990FB81F986CF9091E406892F82
:103D20008F7B96FF80646FCF0E94ED0F9091E40629
:103D3000892F97FB87F9805866CF61E08EE090E08D
:103D40000E94472F62CF60E0F9CF9091E406892F5F
:103D50008F7E94FF806157CF9091E406892F8E7FEC
:103D600090FF816050CF9091E506892F877F93FF68
:103D7000886059CF8272F801E052F847EB30F105C4
:103D800008F05BC0EE55F04D0C94F82E8091DE06E5
:103D90008272F801E054F847EF30F10508F04DC0A9
:103DA000E355F04D0C94F82E81E00E94220A0ACED1
:103DB000811511F10E94690A05CE811511F10E9449
:103DC0008B0A00CE811511F10E94A00AFBCD81154E
:103DD00011F10E94B80AF6CD811511F10E94CE0AA8
:103DE000F1CD0E942B0A81E00E94AD09EBCD0E942B
:103DF000380AF9CF8115F1F20E945F0AE3CD8115EF
:103E0000F1F20E94820ADECD8115F1F20E94940A3D
:103E1000D9CD8115F1F20E94AC0AD4CD8115F1F211
:103E20000E94C40ACFCD811529F00E94EF0ACACDA5
:103E30008115D9F30E94D80AC5CD07378CE718073A
:103E4000F1F008378CE7180729F19801205E324518
:103E50002032310520F5911134C00F7181E090E0DE
:103E600002C0880F991F0A95E2F78C01682F83E042
:103E700090E00E94472F802F0E94B705A3CD81E0DC
:103E8000911551F00E94BD0543E062E081E00E947F
:103E90003A0698CD82E0F4CF0E94C605F5CF911581
:103EA00081F10B358CE7180711F10C358CE71807F9
:103EB00099F00A358CE71807C1F001308CE7180734
:103EC000F1F003308CE71807A1F001151C47C9F485
:103ED0000E94ED0F0E944D0C8091E506002482FFA8
:103EE0000394802D0E94340F6DCD81E0FBCF80E0E4
:103EF000F9CF6FEF7FEF80E090E00E94612F0E948A
:103F0000F80FF70100811181911509F461C0C80112
:103F10000E94F415D82E682FC8010E94D105B8015F
:103F20008D2D0E94E8150E949307182FA92EF701E6
:103F3000C580B680B2948FE0B8228091E306877086
:103F400001F1DC2CC114F1F0892F807F803461F005
:103F5000812F805E8830A8F0892F807E803221F406
:103F6000123078F0B11469F08091E50682FF09C043
:103F700082E00E9481068091E3068770DD24D3945D
:103F80008111D12C8A2D82958F70883009F4EBC075
:103F900020F5823098F1825F8F70823008F467C01C
:103FA000D11409F40FC18091E30680FD0BC1F70124
:103FB00015828695869586950E94BD05C70158DCB9
:103FC0008091E3068695869586950E94C605FAC07F
:103FD000C8010E940706D82EA2CF893009F43EC13D
:103FE0008A5F8F708230E0F6123F09F049C18A2D56
:103FF0008F71C11042C10E94BD05E2C00A2D0F7031
:104000008A2D803110F00295007FC114B9F001159E
:1040100069F0812F805E883010F0111109C0809105
:10402000DE06802B8093DE060E94AF0F812F41C0F9
:104030008091E606802B8093E606F6CF812F0E94C2
:104040000213011509F4ACCF812F805E883010F087
:10405000111104C0802F0E94970606C00095809120
:10406000E60680238093E6060E94AF0F99CF0A2DC3
:104070000F708A2D807F803211F00295007F113001
:1040800040F009F451C0C11409F45CC0B114F9F056
:10409000CDCF8091E50682FD16C0C11469F00115EF
:1040A00039F08091DE06802B8093DE060E94AF0FF0
:1040B00080E00E94AA1274CF80E00E9402130115D2
:1040C00009F46ECFC7CFC114A9F0B11004C0802F7E
:1040D0000E94571365CF8B2D813009F061CF8091FD
:1040E000DF06902F9823091709F45ACF802B80936D
:1040F000DF0656CFB11054CF802F0E9460139091ED
:10410000DF06802F892329F0802F809589238093D3
:10411000DF068091E006902F982309F441CF0095A7
:1041200008230093E0063CCF8B2DC11421F086308C
:1041300008F036CFCCCF853008F032CF802F0E94E8
:1041400060132ECFB114D1F3193349F48FEF97EEEA
:1041500023E0815090402040E1F700C00000812F13
:104160000E9402131DCF8A2D8370E1F5C11028C073
:10417000812F829586958770880F880F412F4F7009
:10418000082E01C0440F0A94EAF7212F207114FF72
:1041900006C02FE001C0220F8A95EAF720958A2DEC
:1041A000869586958370982F8230A1F08330B9F080
:1041B0008091E106913059F0242B82230E94B705AB
:1041C0000E94E60B60E0C7010E9422160ACC842BF5
:1041D000822BF4CF242B8091E1068227EFCF822F10
:1041E000842BECCFC11459F1A0FEEACF812F829528
:1041F00086958770880F880F412F4F70082E01C059
:10420000440F0A94EAF7212F207114FF06C02FE013
:1042100001C0220F8A95EAF720958A2D869586950A
:104220008370982F823091F08330A9F08091E2065C
:10423000913049F0242B82230E94BA05C1CF8230ED
:1042400008F4BECFD3CF842B822BF6CF242B8091C2
:10425000E2068227F1CF822F842BEECF8A2D8F703A
:10426000082FC11431F00E94BD05812F0E94571301
:10427000A7CF812F0E946013802F0E94C605A0CF78
:1042800070F4103FC9F0113F91F0C11409F451C00E
:10429000B11409F44BC0812F0E94AA1291CF133F91
:1042A000F9F0143F91F79091E50692FD26C08A2D12
:1042B0008F71C11411F39FCE8B2DC11479F085300D
:1042C00008F07ECF8A2D8F71282F81E001C0880FE2
:1042D0002A95EAF79091E2068927AECF8630F0CF93
:1042E00080E0C11409F4A8CF8A2D8F71982F81E046
:1042F00001C0880F9A95EAF79FCFC11461F08A2D0B
:104300008F7192FF78CE982F990F990F990F936024
:104310009093E30670CE81E00E9481068B2D82305F
:1043200008F44ECF82E00E9481064ACF8A2D8F7119
:1043300062CEB11479F0193349F48FEF97EE23E090
:10434000815090402040E1F700C00000812F0E9482
:10435000021336CF8A2D8F7190CF8091DE06063101
:104360002CE7120709F006CD8A7A91E0811101C08D
:1043700090E09093DD0665E3811101C069E28AED6A
:1043800092E00E94FC0B0E94AF0F1CCB06318CE721
:10439000180709F0FBCC8091DD0665E3811101C0AF
:1043A00069E28AED92E00E94170CEDCF8091270719
:1043B000803170F480912607811551F0E091E80674
:1043C0002091E70630912207409121072E1301C06A
:1043D0000895BF0187E0E89FF0011124DF01A75194
:1043E000B94F14968C911497811551F111968C91B7
:1043F0001197831325C08C91841322C015968C913C
:10440000159781111DC012968D919D91A091230742
:10441000B09124078A1B9B0B883C910588F48091FE
:1044200027078F70806180932707E151F94F8081C2
:104430008F708061808381E297E01ADA0C947706AE
:104440006F5F7F4FFB01E770C1CFADE0B0E0EBE203
:10445000F2E20C94C62E8C0186E0F801DE0118967B
:1044600001900D928A95E1F7F801F580848191E23F
:10447000892E97E0992E70902507711017C081152D
:1044800091F0F11409F40EC1C8010E944A16811579
:1044900009F408C187E0F801A1E2B7E001900D92AC
:1044A0008A95E1F783DFFF24F39455C0D080A28082
:1044B000B380C09026072091230730912407A501DF
:1044C000421B530BC11409F4BDC0483C510508F010
:1044D00076C0811541F3809122079180E0902707F3
:1044E0009E2D903108F057C0981214C0809121077A
:1044F0008D1110C0F11049C08E2D8F708061809396
:10450000270781E297E0B4D980912707F8018683D5
:10451000F12C21C0F11039C040E0692D8D2D0E9491
:10452000580640E0692D8D2D0E945806F82E811105
:10453000EFCF888599850E943F16292F22952F70ED
:10454000903470F49F70223098F09115A9F0F80122
:104550009681903188F48F2D2D96EDE00C94E22E0B
:104560002A5F2F70223060F0C80182D9FC2CF3CF73
:10457000911511F0811579F3805E883060F3F4CFE6
:10458000803F48F3815F8330F9CF809127078160B6
:1045900080932707BDCF981237C0809121078D11D6
:1045A00033C0F11031C0E682C80162D987E0F8015A
:1045B000A1E2B7E001900D928A95E1F774CFE09007
:1045C00027079E2D903148F481E297E051D9F401FC
:1045D00087E011928A95E9F79BCF811509F463CFA3
:1045E00090912207818198130FC0809121078D112E
:1045F0000BC0F11009C0E682C8013AD9F40187E086
:1046000011928A95E9F74FCFC8010E944A16811589
:1046100009F448C0F11409F445C08E2D803208F425
:1046200039CF809121079091220789839A83AB82A9
:10463000BC827D821E82809127078F83CE010196E6
:1046400017D928CF483C510508F0C1CF811509F48E
:104650002ACFF11439F1909122078181981318C063
:10466000809121078D1114C08091270780FD9ECF76
:10467000803108F49BCF8683807F803F09F494CFFC
:104680008681982F907F905F8F70892B86838CCF47
:10469000C8010E944A168111FDCE809127078160D2
:1046A00080932707C801E4D8FECEABE1B0E0EBE58C
:1046B000F3E20C94CF2E4E8B5F8B688F798F8A8FAD
:1046C000192F9B8F91111092E6061D8A86E0FE013C
:1046D0007696DE011F9601900D928A95E1F70A8D7C
:1046E000011561F00B8B1C8B61E0CE010F960E94CF
:1046F000221661E0CE010F960E9422160B8B1C8BB6
:1047000087E0FE013F96DE01189601900D928A9592
:10471000E1F7CE01089699DE81112EC02091E706BF
:104720003091E80687E0AE01485F5F4FFA014750DD
:104730005109DA0101900D928A95E1F78C85811576
:10474000D9F0822F90E08395877090E0AC01341708
:104750001506E1F097E0929FD0011124A751B94FBF
:104760009E012F5F3F4FF90101900D929A95E1F75D
:104770004093E7060E9477068091E8069091E7064D
:10478000891311C06B96E4E00C94EB2E0E94ED0FA0
:104790001092E7061092E806E1E2F7E087E0119256
:1047A0008A95E9F7E9CF27E0829FC001112487515C
:1047B000994F4BDE811531F38091E8069091E9061F
:1047C000019687708093E806D7CFA6E0B0E0EBEEC5
:1047D000F3E20C94CF2E0E94F3198C018091B40661
:1047E0009091B5068017910771F019821A820E9484
:1047F000F319BC0149815A8180E090E056DF0093B3
:10480000B4061093B5062696E4E00C94EB2ECDB7D3
:10481000DEB7A4970FB6F894DEBF0FBECDBF85B745
:10482000806885BF85B7806885BF84B7877F84BF70
:104830000FB6F894A895809160008861809360001D
:10484000109260000FBE80E890E00FB6F89480935D
:104850006100909361000FBE81E0809311018AE6B0
:1048600098E08093D8029093D9020E948D0D0E9407
:104870003E0D8091E20084608093E2007894809104
:104880003A06811599F08091E9001091EC008F7043
:1048900010FB112717F9182B1092E9008091E800FE
:1048A00083FD0E9404101F701093E90082E084BD14
:1048B00093E095BD9AEF97BD80936E001092B0067D
:1048C0001092B1061092B2061092B3060E94A01682
:1048D000811102C00E943B198091D80080618093B1
:1048E000D8008AE18A95F1F700C08091D900182F8D
:1048F000117080FD04C00E948D0D10923A06109335
:10490000AE060E94B716811102C00E9461198EE0A6
:1049100090E00E942B2F811529F060E08EE090E05E
:104920000E94472F8EE090E00E942B2F91E0811192
:1049300001C090E09093AF06909312018091AE0673
:1049400081110E945E2D8091AF0690E0811101C01F
:1049500095E09093A30685E0891B809395066CEC07
:10496000E62E62E0F62E01ED12E0F70181917F0163
:104970008F3F11F00E946C080E151F05B1F751ED25
:10498000E52E52E0F52E07ED12E0F70181917F014F
:104990008F3F11F00E946C080E151F05B1F7E9E971
:1049A000F6E08AE011928A95E9F7E4EAF6E08AE017
:1049B00011928A95E9F70E94B716811102C00E94F0
:1049C000611982E090E00E942B2F8093F90384E02C
:1049D00090E00E94332F8093E4069093E5060E94B6
:1049E000081A8FEF96E721E0815090402040E1F7D0
:1049F00000C000000E94081A8091990680FF08C03C
:104A00006FEF7FEF80E090E00E94612F0E944D0CDD
:104A100083E090E00E942B2F0E94B7050E94590B63
:104A200081E08093EB0348E050E067E170E082E3CF
:104A300096E00E941B2F1092EB0380913206843087
:104A400010F40E94CC1683E08093260680E28093C7
:104A5000EC03CFD66BE070E087E894E00E948B19FE
:104A60008115E9F18091260665E070E081FD0EC1B7
:104A700082E894E00E948B19811589F16DE070E065
:104A800080E794E00E948B19811549F10E94260C61
:104A9000DC01CB01805A9541AF4FBF4F80932A066E
:104AA00090932B06A0932C06B0932D06E6E2F4E03B
:104AB000DF0180E092E01D920197E9F7E0930404A2
:104AC000F09305048FEF9FEF8093280690932906BB
:104AD00081E08093300680933F06109227068091F4
:104AE000AE06811101C0EDD78EEA92E080933A07BD
:104AF00090933B0784E080933907AEEAB2E020E070
:104B000013968C911397811501F12830F0F4822FC0
:104B100090E0FC01EE0FFF1FE85DF84F8F0100975A
:104B200061F0F801529142918F01FA01348114969B
:104B30006C911497631708F4ACC0880F991F885DB7
:104B4000984FFC01A083B1832F5F159682E0A23CB1
:104B5000B807B1F6209338078091E2060E94AB0DAA
:104B600083E191E08093B6069093B70691E0C92E59
:104B7000D12C80913A06853069F400E110E482E19D
:104B8000F82E80913A06853009F488C00E94ED0F16
:104B90000E94E60B0E94081AAAEFAA2EA3E0BA2EE2
:104BA000B9E98B2EB6E09B2EF401D5019D91808151
:104BB00024E0A430B20709F4CCC031969817B1F3C1
:104BC0002090AE06FFEEEF2EF3E0FF2E712CF401E5
:104BD00061904F01F50141905F01461409F441C015
:104BE000462400E010E055245394842D852189F15A
:104BF000362C35202114F9F0F701808190E09601E0
:104C0000002E01C0220F0A94EAF78223892B99F41F
:104C100009837A820E94F3198B839C8381E08D83C0
:104C200091E0311001C090E09E8349815A816B81EF
:104C30007C818D813ADD31100CC08C2D002E01C09D
:104C4000880F0A94EAF7982F9095F70180818923BD
:104C50008083550C0F5F1F4F0630110531F6F501AB
:104C6000629273948FEFE81AF80A872D8A3009F060
:104C7000AECF0E94320C60938D0670938E068093A7
:104C80008F0690939006BB24B39467C08DE794E0A1
:104C9000F1CE0197F8014283538341CF80913A06C8
:104CA000843039F10E94E2160E94BB191092ED0384
:104CB00088E190E00FB6F894A895809360000FBE4D
:104CC0001093600083B7817F846083BF83B7816066
:104CD00083BF7894889583B78E7F83BF0FB6F8948F
:104CE000A8958091600088618093600010926000B8
:104CF0000FBE0E94081AE9E9F6E0AFEEB3E080E0EB
:104D000021912D9391E0211101C090E0892B96E033
:104D1000E33AF907A9F7811509F433CF8091EE033F
:104D2000811509F42ECF09BDF9BC09B400FEFDCFF1
:104D30008091D8008F7D8093D8008091E0008260C0
:104D40008093E0008091E00081FDFCCF0E94ED0F98
:104D500018CF981335CF39DDB12C8091AE0681156F
:104D600031F1E090D806F090D906E114F104F9F0A1
:104D70000091DA061091DB060E94F319801B910B5B
:104D8000893C9105A0F00EE611E0E11411F000E07D
:104D900010E060E08E2D0E94970B009741F0FC011F
:104DA000258122FD04C0BC01C8010E9495130E9408
:104DB000E21680913006811509F47CC000912E0620
:104DC00010912F060E94F319801B910B819708F414
:104DD0004FC00E94F31980932E0690932F0680E017
:104DE0000E94090B8091E2060E94AB0D8091AF06F4
:104DF000811509F4B1C080E00E94090B60E670E003
:104E000082E796E00E941A0B83E00E94090BE09172
:104E10000404F0910504CF0186529440AF01465E30
:104E20005240413022E0520710F040E052E0209121
:104E30002806309129067F01ACE3B7E08417950777
:104E400008F46EC020932806309329068DE00E9456
:104E5000090B60E470E082E196E00E941A0B8FE09B
:104E60000E94090B60E270E082E596E00E941A0B56
:104E70008091280690912906892B09F08EC0809197
:104E80003F068115B9F00E94260C00912A06109168
:104E90002B0620912C0630912D06DC01CB01801BC6
:104EA000910BA20BB30B8F3F9F4FAF4FBF4710F437
:104EB0000E94BB19B1100E9498190E94E60B9091B4
:104EC0003106891721F0809331060E94260C8091CB
:104ED0003A06843009F04DCE83E08093E90080915A
:104EE000E80082FF46CE8091E80090E085FF06C092
:104EF0000E940D0D811509F428C191E08091E80010
:104F00008B778093E800911509F433CE8981E82FDF
:104F1000E150E33108F043C1F0E0E454F04D68C7DC
:104F20001D91F70161917F011617A1F0BF0161503A
:104F30007109FB011083BC01E5E076956795EA9560
:104F4000E1F7F60102C0EE0FFF1F6A95E2F7BF011D
:104F50002E2B372B019672CF0E94E60B02E315E051
:104F600081FD02C002E914E080E00E94090B60E6C6
:104F700070E082E796E00E941A0B84E00E94090B21
:104F800060EA70E0C8010E941A0B8DE00E94090BD4
:104F900060E470E082ED95E069CF80913006811584
:104FA00009F46DCF80912706811169CF0E9498196D
:104FB00041E1E42EF12C209128063091290621159B
:104FC000310509F45CCFEA9411F459CFF3948F2D95
:104FD00090E026010F2C02C0440C551C0A94E2F705
:104FE000A20142235323452B89F32091260620FD5D
:104FF00042C09695879596958795482F282F9F2D87
:105000009295990F9076392F315E842F90932101DC
:1050100080932401309322012093250124E630E07F
:1050200047E050E06FE171E088E716D4892B09F082
:1050300026CF80E2F89E300111248091260680FD63
:1050400023C0A3014A5D5B4F04E610E020E230E09C
:1050500060E488E791D4892B09F011CF40945094F3
:105060008091280690912906842195218093280615
:1050700090932906A0CF9F2D990F990F990F392F43
:10508000395F80E023E0C2CFE6E0F4E080E21192F5
:105090008A95E9F786EC92E089A39AA322EC222E66
:1050A00022E0322E6AEC72E0A9A1BAA1ED91A9A387
:1050B000BAA3D1018D911D01282F260D372D311D49
:1050C0002BA33CA3F0E0EA5FFB4F20E030E097E049
:1050D000892E821AAC2C022E01C0AA0C0A94EAF77F
:1050E0000BA11CA10A5D1B4F90E0D8018D918D0191
:1050F0008A21482D491B477050E0A82F042E01C07B
:10510000AA0F0A94EAF7519541955109477001C0D9
:1051100086954A95EAF78A2B4081482B40839F5F0A
:10512000983019F72F5F3F4F31962830310579F6C7
:1051300089A19AA16817790709F0B6CF04E610E0B3
:1051400020E230E046E054E083CF80E2E82EF12C0C
:105150008E010F5F1F4F8091E80085FD0AC080918E
:10516000E8008B778093E8000E940D0D811599F37C
:10517000C4CE8091F100F801808381E0E81AF10843
:1051800009F4BBCEE6CF1A828CE08B8319C08A81EA
:10519000833081F138F4813029F1823051F08FEF82
:1051A00089830EC08430D9F71B821C821D821E8227
:1051B00007C088E290E04FD61B821C821D828E833E
:1051C000E091B606F091B706309709F4D2CC02848C
:1051D000F385E02D309709F4CCCC60E2CE01019646
:1051E0000995C7CC0E94260C09D66B837C838D83DE
:1051F0009E83E6CF8B8190E0FE0134968A30910544
:10520000FCF611920196FACF8A81823031F0853016
:1052100031F680E00E94220AD3CF6B817C818D81A0
:105220009E81ECD588E290E032D6CACF4C816B816A
:105230008A810E94BE159827892798278D839E838F
:10524000BFCF2D813E813227232732274C816B81AE
:105250008A810E944B0FB4CF0E94710FB1CF9A8107
:10526000933009F09CCF883009F439C0893009F4B3
:1052700062C08B81833061F158F4813091F08230CB
:1052800009F09ECF8C8181111CC00E94380A98CFF2
:10529000843009F095CF8C8120E0409135066D81F6
:1052A0000CC04C8128E7429F040E40E0411D1124B0
:1052B0008091330620E06091340690E00E94720AEB
:1052C0007FCF0E942B0A60E08C810E94440A78CF35
:1052D0008C818093360680E00E94AD0971CF8B816E
:1052E000833031F170F48130B1F0823009F068CF51
:1052F00080913206982F9370C9F0869586958C839D
:105300005FCF843009F05CCF809133068C8380912D
:1053100034068D8355CF809135062FEF829FC001D3
:10532000112468E770E019D56C834ACF80E0E7CF9D
:1053300080913606E4CF0E94C11642CF80E18A8375
:105340003FCF81E08A8387E020CF8A809B809824AA
:1053500089249824A12CB12C8E010F5F1F4FEC8063
:10536000E00EF12EF11C0E151F0509F429CF87E080
:10537000881681E09806A104B10470F4C401875036
:105380009D4F69D5F80184830F5F1F4F8FEF881AF7
:10539000980AA80AB80AE7CF80E0F4CFFC808A8098
:1053A0009B80982489249824A12CB12C8E010F5F16
:1053B0001F4F250132014F1451046104710408F09C
:1053C000FFCE87E0881681E09806A104B10430F48E
:1053D000F8016481C40187509D4F59D58FEF481A59
:1053E000580A680A780A8FEF881A980AA80AB80A31
:1053F0000F5F1F4FE0CF0E940019E2CE86E09FCFE3
:10540000FC808A809B80982489249824A12CB12C2C
:10541000250132018E010B5F1F4F4F1451046104AF
:10542000710408F0CDCE80ED881682E09806A104C4
:10543000B10488F4C40189960ED5F80181938F01D7
:105440008FEF481A580A680A780A8FEF881A980A64
:10545000A80AB80AE2CF80E0F0CFFC808A809B8067
:10546000982489249824A12CB12C8E010F5F1F4F02
:10547000250132014F1451046104710408F0A0CEDB
:1054800080ED881682E09806A104B10428F4F801A2
:105490006481C4018996FBD48FEF481A580A680AC0
:1054A000780A8FEF881A980AA80AB80A0F5F1F4F68
:1054B000E1CF78941F921FB61F9211248F939F9370
:1054C000AF93BF938091F5029091F602A091F702FD
:1054D000B091F8020196A11DB11D8093F502909341
:1054E000F602A093F702B093F802BF91AF919F919B
:1054F0008F911F901FBE1F9018951F920F920FB68D
:105500000F9211242F933F934F935F936F937F9349
:105510008F939F93AF93BF93EF93FF938091E1009D
:1055200082FF09C08091E20082FF05C08091E10006
:105530008B7F8093E1008091DA0080FF24C080910E
:10554000D80080FF20C08091DA008E7F8093DA003F
:105550008091D90080FFA9C080E189BD82E189BD29
:1055600009B400FEFDCF81E080933A068091E40209
:10557000811109C00E948D0D0E943E0D8091E200B4
:1055800084608093E2008091E10080FF1AC08091E6
:10559000E20080FF16C08091E2008E7F8093E200DF
:1055A0008091E20080618093E2008091D800806267
:1055B0008093D80019BC85E080933A0683E08093FD
:1055C00011018091E10084FF2FC08091E20084FFEF
:1055D0002BC080E189BD82E189BD09B400FEFDCF09
:1055E0008091D8008F7D8093D8008091E1008F7EDC
:1055F0008093E1008091E2008F7E8093E2008091B1
:10560000E20081608093E2008091E302811509F459
:1056100052C084E080933A0680913A06843009F0C3
:1056200052C082E0809311018091E10083FF2CC081
:105630008091E20083FF28C08091E100877F809302
:10564000E10082E080933A061092E3028091E1004B
:105650008E7F8093E1008091E2008E7F8093E20054
:105660008091E20080618093E20042E060E080E0AF
:105670000E94BE0C8091F00088608093F00081E071
:105680008093110180931001FF91EF91BF91AF9131
:105690009F918F917F916F915F914F913F912F914A
:1056A0000F900FBE0F901F90189519BC10923A06DC
:1056B0001092E40268CF8091E30087FF02C083E08C
:1056C000A9CF81E0A7CF81E0ADCF1F920F920FB697
:1056D0000F9211241F932F933F934F935F936F93D8
:1056E0007F938F939F93AF93BF93CF93DF93EF936A
:1056F000FF93E9EEF0E080811091EC008F7010FBD9
:10570000112717F9182B1082C0EFD0E08881877F0E
:10571000888378940E940410E9EEF0E0108288817A
:10572000886088831F701083FF91EF91DF91CF9184
:10573000BF91AF919F918F917F916F915F914F91A9
:105740003F912F911F910F900FBE0F901F901895B2
:10575000EF92FF921F93CF93DF93182FEB011092DC
:10576000BC0084EA8093BC000E94F3197C01809104
:10577000BC0087FF26C08091B900887F883029F05F
:105780008091B900887F803189F51093BB0084E84F
:105790008093BC000E94F3197C018091BC0087FFBC
:1057A0001EC02091B900287F80E090E0283189F068
:1057B00081E090E0203409F480E091958195910991
:1057C00008C0C7010E94FF19C817D90780F68EEFDD
:1057D0009FEFDF91CF911F91FF90EF900895C70148
:1057E0000E94FF19C817D907C0F6F1CF8FEF9FEFBE
:1057F000F0CF1092B9008CE08093B80008950F9319
:105800001F93CF93DF93EB018093BB0084E88093D9
:10581000BC000E94F3198C018091BC0087FF10C06E
:105820002091B900287F81E090E0283209F480E0DF
:10583000919581959109DF91CF911F910F910895D5
:10584000CF3FDC0749F3C8010E94FF19C817D907E9
:1058500018F78EEF9FEFEFCFA0E0B0E0E1E3FCE2BE
:1058600095C2982E862E772E6A0179010E94F3192F
:105870005C0184E1E816F10410F18FEFE816FE04F4
:1058800009F1C70164E170E068D2162F072F612F7C
:10589000702F892D5DDFEC01892BB1F4082D172DB8
:1058A000C00ED11E0C151D0511F02097C1F084E922
:1058B0008093BC00CE01CDB7DEB7EDE083C211E02E
:1058C00000E0E5CF15E0FCCF8FEFE816FE04F9F21B
:1058D000C5010E94FF19E816F906C8F6DFCFB70127
:1058E000F80181918F018BDFEC01DCCFA0E0B0E00B
:1058F000EBE7FCE24BC2982E862E772E6A018901D7
:105900000E94F3195C010431110500F10F3F1007EB
:1059100001F1C80164E170E020D2EB01BE01892DE4
:1059200017DF7C01892BB9F4C82DD72DCC0EDD1ED5
:10593000CC15DD0519F0E114F104B9F084E9809388
:10594000BC00C701CDB7DEB7EDE03CC2C1E0D0E09E
:10595000E5CFC5E0FCCF0F3F100701F3C5010E9462
:10596000FF1908171907D0F6DFCFFE018491B8019F
:1059700046DF7C012196DCCFA0E0B0E0E1ECFCE268
:1059800004C2982E862E742E652E6901E8010E94AD
:10599000F3195C010431110508F10F3F100711F1F3
:1059A000C80164E170E0D9D1F62EE72E6F2D7E2D6F
:1059B000892DCEDE8C01892BC1F0CF3FDC07B1F3FE
:1059C000C5010E94FF19C817D90780F784E98093A1
:1059D000BC00C801CDB7DEB7EEE0F3C1FF24F394FD
:1059E000E12CE4CF85E0F82EFBCFBE01882D07DF48
:1059F0008C01E72CF62CCE0CDF1CEC14FD0431F3EB
:105A00000115110519F7BE01F70181917F01F7DE3C
:105A10008C01F3CF8EE14A9B02C08150E1F74A9B93
:105A2000FECF08955A9880E28A95F1F75A9A089520
:105A3000FC018BE08A95F1F728E080E090E031E00E
:105A400040E14A95F1F7880F4A9B02C08160932795
:105A500042E04A95F1F7000040E14A95F1F7215004
:105A600079F720E12A95F1F729B132E03A95F1F77B
:105A7000000030E13A95F1F731E022FD93272081D3
:105A8000920F90830895A1E0B0E0E8E4FDE285C1C3
:105A900019828C017C01E60EF11CBCDFCE0101965F
:105AA000C7DFF80181938F01EE15FF05B1F781E0A3
:105AB0009981911180E02196E6E08BC1529A5A9A21
:105AC000089552985A9AEA9AE9E6F0E080818F7C2C
:105AD000808308956150770B91E001C0990F6A951A
:105AE000EAF7692F90E021E0611108C0911591F06B
:105AF0005A9A80E28A95F1F75A980895362F3823FA
:105B000039F05A9A922730E23A95F1F76695ECCF40
:105B10005A98F9CF5A98EDCFFF920F931F93CF93D6
:105B2000DF93EC018C01060F111D8991F82E7ADFAD
:105B300068E08F2DCFDFC017D107B9F7CDB7DEB73B
:105B4000E5E048C11F920F920FB60F9211240F93F8
:105B50001F932F933F934F935F936F937F938F93F5
:105B60009F93AF93BF93EF93FF93CF93DF930F92E6
:105B7000CDB7DEB719824EDFCE01019659DF082F6F
:105B8000069506950695282F22952570902F9570DD
:105B9000920F292F237096959695920F98279770BC
:105BA0008981892B09F055C00A3008F052C080E184
:105BB0008A95F1F75A9A529A82E08A95F1F700C0D5
:105BC0005A9888E0089F80011124D801AA5DBE4F31
:105BD0001696ED91FD911897309791F06091CA0259
:105BE0007091CB0214962D913D91260F371F15977A
:105BF0008D919D91680F791F4C9113978C91099508
:105C0000F801EA5DFE4F6381611549F02091CA02F7
:105C10003091CB0284819581820F931F7DDF02DF5B
:105C200080E18A95F1F75A9852985A9A80E18A95BC
:105C3000F1F7F801EA5DFE4F6081611549F02091AE
:105C4000CA023091CB0281819281820F931F1BDFA8
:105C5000E1DE0F90DF91CF91FF91EF91BF91AF9176
:105C60009F918F917F916F915F914F913F912F9174
:105C70001F910F910F900FBE0F901F9018950F93CB
:105C80001F93CF93DF93EC010A970CF05EC0F8945A
:105C9000529A5A9885E08A95F1F700009C2F9695C4
:105CA00095708C2F8570980F892F83709695969597
:105CB000292F93E0CC0FDD1F9A95E1F7280F822F53
:105CC0008C2B082FAFDE00C068E0802F03DF80E15F
:105CD0008A95F1F752985A9A4A9B30C087E090E033
:105CE0004A992EC0FE01EA5DFE4F6381611559F0AD
:105CF0002091CA023091CB0284819581820F931F3B
:105D0000C2DE8115F9F086DE80E28A95F1F75A98B5
:105D1000529A80E18A95F1F7CA5DDE4F688161157C
:105D200049F02091CA023091CB0289819A81820F79
:105D3000931FF2DE77DE789481E008C000C0CCCFFC
:105D4000019749F4529A5A9A789480E0DF91CF9162
:105D50001F910F91089500C0C3CFAA1BBB1B51E137
:105D600007C0AA1FBB1FA617B70710F0A61BB70BCB
:105D7000881F991F5A95A9F780959095BC01CD0170
:105D800008952F923F924F925F926F927F928F92DF
:105D90009F92AF92BF92CF92DF92EF92FF920F93BA
:105DA0001F93CF93DF93CDB7DEB7CA1BDB0B0FB6C4
:105DB000F894DEBF0FBECDBF09942A883988488881
:105DC0005F846E847D848C849B84AA84B984C88417
:105DD000DF80EE80FD800C811B81AA81B981CE0F0E
:105DE000D11D0FB6F894DEBF0FBECDBFED010895F3
:105DF000EE0FFF1F0590F491E02D09946927962777
:105E000069277827872778270895FB01DC0104C0DC
:105E10008D910190801921F441505040C8F7881BA2
:105E2000990B0895FB01DC0102C001900D924150D5
:105E30005040D8F70895DC01CB01FC01F999FECF61
:105E400006C0F2BDE1BDF89A319600B40D92415002
:105E50005040B8F70895F999FECF92BD81BDF89AE8
:105E6000992780B50895A8E1B0E042E050E0E5CF81
:105E7000DC01A40FB51F4150504040F0CB01840F0E
:105E8000951F2E9105D041505040D8F70895262FE8
:105E9000F999FECF92BD81BDF89A019700B4021620
:105EA00039F01FBA20BD0FB6F894FA9AF99A0FBECE
:105EB00008950396272FECDFEADF252FE9DF242F53
:105EC000E7CF0196272FE4DFE2CFF894FFCFE11070
:105ED00007110D1107110D115B117D110D116C12C0
:105EE00079125817811797179A179D17A0171F181F
:105EF0005D18441EAC1E4C1E161E1A1E501E1E1E81
:105F0000541E601E2A1EA51E2E1E641E321E681EF2
:105F10008D1E361E6C1E941E3C1E721E7A1E221E84
:105F2000581E261E5C1E401E761E841E9D1EA31E2D
:105F3000101E481EB31EED1DF11DE41DE91DF51DCB
:105F4000F91DFD1DD41ED81EFA1EDD1EFF1EE21E09
:105F5000041FE71E091FEC1E0E1FF11EF71ED41EA4
:105F6000D81EFA1EDD1EFF1EE21E041FE71E091FBB
:105F7000EC1E0E1F131F181FC328C728042916293B
:105F800021292C292F292F292F29CF28CF289E29B5
:0E5F9000A129A529CE29FB29FE29002A2D2AA8
:105F9E00E10039004700FFFF0300FF003905000054
:105FAE00010001230C210F5E0C5F0C600C190F0019
:105FBE0021007F220003000000010000000000000D
:105FCE000005010000000506000000000000040BA3
:105FDE00000000000000010F000000000000011092
:105FEE00000000000000011100000000000001127E
:105FFE000000000000000C13000000000000EE1274
:10600E00FE12321300000001FF00FF78FF050200B0
:10601E00000102030405060708090A0B0C0D0E0FFA
:10602E001011121314151617FF18191A1B1C2827F6
:10603E00262524232E2D2C2B2A2934333231302F92
:10604E003A3938373635FF3F3E3D3C3B00000F00B6
:10605E001E002D003C004B0000100F101E102D10C6
:10606E003C104B1000200F201E202D203C204B20DA
:10607E0000300F301E302D303C304B301E402D4046
:10608E003C404B405A400F142D144B140F2D2D2D08
:10609E004B2D9500A400B300C200D100E000951076
:1060AE00A410B310C210D110E0109520A420B3207C
:1060BE00C220D120E0209530A430B330C230D13090
:1060CE00E03086409540A440B340C2409514B314CE
:1060DE00D114952DB32DD12D04040404040404040D
:1060EE000404040404040404040404040404040462
:1060FE00040404040402020202020204040404045E
:10610E000404040404040404040404040404040441
:10611E000404040404040404020202020202003114
:10612E0031295A1B750A42415345004C4F5745526F
:10613E000052414953450041444A5553540000967C
:10614E00020101019B02010202A102010003A7024A
:10615E000103000810181810080061066697C6346F
:08616E0035F6F731333236003B
:00000001FF
